:100000000C9472000C948D000C948D000C948D0057
:100010000C948D000C948D000C948D000C948D002C
:100020000C948D000C948D000C948D000C948D001C
:100030000C948D000C948D000C948D000C948D000C
:100040000C948D000C948D000C948D000C948D00FC
:100050000C948D000C948D000C948D000C948D00EC
:100060000C948D000C948D000C948D000C948D00DC
:100070000C948D000C948D000C948D000C948D00CC
:100080000C948D000C948D000C948D000C948D00BC
:100090000C948D000C948D000C948D000C948D00AC
:1000A0000C948D000C948D000C948D000C948D009C
:1000B0000C948D000C948D000C948D000C948D008C
:1000C0000C948D000C948D000C948D000C948D007C
:1000D0000C948D000C948D000C948D000C948D006C
:1000E0000C948D0011241FBECFEFD1E2DEBFCDBF37
:1000F00000E00CBF84B78093000214BE0FB6F894E2
:10010000A8958091600088618093600010926000E3
:100110000FBE0E94F0000C9430010C9400008093FC
:1001200008010895A8E0B1E08C93EBE0F1E0808154
:100130008D7F808361BB8081877F80838AE08A9501
:10014000F1F700C08081886080831C92808182608A
:10015000808311BA089563E883E00E94920063E00F
:1001600080E00E94920060E081E00E94920063E0E3
:1001700083E00E94920061E480E00E9492008FE39D
:100180009CE90197F1F700C0000062E480E00E9462
:1001900092008FE39CE90197F1F700C0000061E253
:1001A00080E00E9492008FE39CE90197F1F700C084
:1001B00000006DE080E00E9492008FE39CE90197CF
:1001C000F1F700C000006AE080E00E9492008FE337
:1001D0009CE90197F1F700C0000090E080E00895ED
:1001E000F8948FEF80BB8093070180930A0111BAC6
:1001F0001092080110920B0180910B018260809394
:100200000B0180910B01846080930B0180910B01A5
:10021000886080930B0180910B01816080930B01BA
:100220008FE891E00197F1F700C0000080910B0189
:100230008E7F80930B018FE99FE00197F1F700C05B
:100240000000789488E19EE00FB6F894A89580931A
:1002500060000FBE90936000A8950E94AB00FCCF99
:04026000F894FFCF40
:00000001FF
